:020000040000FA
:100000003728FF3FFF3FFF3FF000030EF1000408D9
:10001000F2000A08F30083018A010C1910280F2846
:1000200083010C11B01C1B28231C192885110515F0
:100030001B2805118515301C2C283010B108031918
:100040002428A621B0142C28851105110330960010
:10005000FF309500B0102C282D28A30A73088A00C1
:1000600072088400710E8300F00E700E0900830187
:100070008A018B01640000308500FE308600073065
:100080009F008316CF30810021308500003086002C
:10009000831283018E018F0101309000033096009E
:1000A000FF30950095000B30970083018316F930DF
:1000B000920083124D3092008301831633309900F1
:1000C000043098008312103098008301A201A3012C
:1000D000B001B1010230B200B301B401B501B60103
:1000E000B701E001E101E201E301E401E501E6011C
:1000F000BD01BE01BF01C201C301C001AA30C100E0
:10010000BC000A30B8006430B9003C30BA0001309D
:10011000BB006430E8005530E9004630EA00373073
:10012000EB002830EC001930ED000A30EE008301BE
:100130008C01831604308C008301C0308B000518BD
:10014000B02830169730BE00BD1700309522B7009A
:10015000B5000430B400B600B3000F30B100301465
:10016000830147228C18B6288E22B0288C10640098
:10017000A20A830135080319FB283D18F228BD188F
:10018000F228B40BFB283308B400B60BFB28350368
:1001900037020319F2283019D5280030B100301485
:1001A00030150130B400B600FB283011B50A35080F
:1001B00095228A01A0000F39B1003014200E0F39AA
:1001C000B6003308B40031080319F1280739A0003C
:1001D000073C0319A0012008603E840064308000C1
:1001E000BC01FB28B1013014B501B401B601B30163
:1001F000B7013D10BD10830122080139031D4729B5
:10020000BC1806296008031DE0030A296008643C45
:10021000031DE00A3C1910296108031DE10314299C
:100220006108643C031DE10ABC191A296208031D18
:10023000E2031E296208643C031DE20A3C1A2429D9
:100240006308031DE30328296308643C031DE30AD4
:10025000BC1A2E296408031DE40332296408643C97
:10026000031DE40A3C1B38296508031DE5033C29EE
:100270006508643C031DE50ABC1B42296608031D92
:10028000E60346296608643C031DE60A00002B22AB
:10029000B80B7F290A30B80083013508031D652992
:1002A0003D185529B019552965293D10B011320A5C
:1002B0000739B20000309522B70001309522B30013
:1002C0000130B5000130B400B60083013508031DCC
:1002D0007F29BD186C297F29BD103F0A0139BF0055
:1002E00000309522B700B5000430B400B600B3006A
:1002F0003F0AA0000310A00D200DB1003014B90B6F
:10030000A5296430B9003508031D9B293F1895299C
:100310000D2240080739A0000130A1000310A10DF3
:10032000A00B8E292108BC069B293A1C9B290D2273
:100330004008BC009B29BA0BA5293C30BA00BB0B76
:10034000A5293C30BB00301EB015B028B10BAD293B
:1003500003309600E73095000C2AB10BB429033026
:100360009600AF3095000C2AB10BBB2903309600E4
:100370007A3095000C2AB10BC22903309600483020
:1003800095000C2AB10BC92903309600193095004D
:100390000C2AB10BD02902309600EC3095000C2AC3
:1003A000B10BD72902309600C23095000C2AB10B50
:1003B000DE29023096009A3095000C2AB10BE5290F
:1003C00002309600753095000C2AB10BEC290230F2
:1003D0009600523095000C2AB10BF329023096009A
:1003E000303095000C2AB10BFA29023096001130FA
:1003F00095000C2AB10B012A01309600F3309500CC
:100400000C2AB10B082A01309600D73095000C2A2F
:1004100001309600BC30950008000830A00040086C
:10042000C2004108C300C20CC30DC30DC30D01308F
:10043000C205C30542084305A100C209C309013032
:10044000C205C30542084305A104A10CC00DC10D9E
:10045000A00B0F2A080005183A2A3E080311973C02
:10046000031DBE0A3E080311963C0319BD1403196F
:10047000BD17462A3E080314053C0318442ABD1B39
:10048000442A3D14BD17462ABE01BD130800E80BDF
:100490004D2A86146430E800512A68086002031867
:1004A0008610E90B572A06156430E9005B2A6908B3
:1004B000610203180611EA0B612A86156430EA000E
:1004C000652A6A08620203188611EB0B6B2A06166E
:1004D0006430EB006F2A6B08630203180612EC0B02
:1004E000752A86166430EC00792A6C0864020318B9
:1004F0008612ED0B7F2A06176430ED00832A6D0803
:10050000650203180613EE0B892A86176430EE0085
:100510008D2A6E0866020318861308000830A000B2
:1005200000000000A00B902A0800A0003208013E45
:10053000A100A10B9C2A002CA10B9F2A782CA10BB7
:10054000A22ABD2CA10BA52A002DA10BA82A3E2D65
:10055000A10BAB2A732DA10BAE2AC42D002EFF3F99
:10056000FF3FFF3FFF3FFF3FFF3FFF3FFF3FFF3F9B
:10057000FF3FFF3FFF3FFF3FFF3FFF3FFF3FFF3F8B
:10058000FF3FFF3FFF3FFF3FFF3FFF3FFF3FFF3F7B
:10059000FF3FFF3FFF3FFF3FFF3FFF3FFF3FFF3F6B
:10080000830104308A0020088207713416341A34B8
:100810001A342A341A341A342A341A341D34163449
:1008200018344A341B341B342B341A341A342A3407
:100830001834183418341A3428342D341A341A342D
:100840002A341A341A342A341A341D34163418341B
:100850004A341B341B342B341A341A342A341D34D2
:100860001B341A341834463411341A3418341634FC
:10087000413411341A3418341634433413341B34CD
:100880001A3418341D341D342D341F341D341834DB
:1008900019344A3411341A341834163441341134AA
:1008A0001A3418341634433413341B341A341834BD
:1008B0001D341D342D341F341D341B34183426349C
:1008C0002D341A341A342A341A341A342A341A3485
:1008D0001D34163418344A341B341B342B341A3468
:1008E0001A342A341D341B341A34183446348034F4
:1008F000830104308A00200882073E340D342734F7
:10090000263444342634273429344B342D344E34A1
:100910002E342D342B3446342B344B342B342934A1
:10092000473424342234C43427342634443426341F
:10093000273449342B342D344E342E342D342B347B
:1009400046341B341B344B342B342934273446347F
:100950002434C2342E342D342B34663426342434DB
:1009600022342434C6342E342D342B3466342634C9
:10097000243422342234A2348034830104308A00A7
:100980002008820729340D34613444342C34CD34AA
:1009900028342B34293444342334C234623444346C
:1009A0002634C83426342434233444342E34CD340D
:1009B000613444342C34CD3428342B342934443439
:1009C0002334C234623444342634C83426342434C4
:1009D000233444342B3489348034FF3FFF3FFF3FBE
:1009E000FF3FFF3FFF3FFF3FFF3FFF3FFF3FFF3F17
:1009F000FF3FFF3FFF3FFF3FFF3FFF3FFF3FFF3F07
:100A0000830105308A0020088207373412344334CA
:100A100026346D344B342634643443342334233445
:100A20002434263468346634433426346D344B34ED
:100A30002634643443342634263428342A346B3440
:100A40004B3420344D3426342A342834263443346D
:100A500026346B3448342B344D342B346A346634AA
:100A6000433426346D344B342634643443342634D2
:100A7000263428342A346B346B34803483010530B7
:100A80008A00200882072E341A3438341A34283465
:100A9000653438341A34283465344F342F346C3488
:100AA0004D342D3468344A342A343D341C342A34CD
:100AB00038341A34283465344A342A343D341C34EA
:100AC0002A3438341A34283465344F342F342F34D0
:100AD0002F342C34BD342D34283425342834263496
:100AE000233461348034830105308A002008820772
:100AF0004A341C3423342834273428342A34253407
:100B00004A3428342734253427348834233428348D
:100B1000273428342A3425344A34283427342534D9
:100B2000273488342C342C341C343C342C342C346E
:100B30004C342C342A3428342A348C342C342C343D
:100B40002D342C342A3425344A342834273425349F
:100B50002734683420342C342C341C343C342C346A
:100B60002C344C342C342A3428342A348C342C340D
:100B70002C342D342C342A3425344A342834273468
:100B80003C341A3488348034830105308A002008CC
:100B9000820725341334153419341A344C34103484
:100BA000153419341A344C341034153419341A34B9
:100BB0002C34293425342934473410341934193469
:100BC00017343534153429342C341C344A341A344F
:100BD00019341A342C34293425342734453440341C
:100BE000FF3FFF3FFF3FFF3FFF3FFF3FFF3FFF3F15
:100BF000FF3FFF3FFF3FFF3FFF3FFF3FFF3FFF3F05
:100C0000830106308A00200882073E3415342434DC
:100C10002D342B3429342B34293426342434813494
:100C200024342D342B342934293428342934AB345A
:100C300024342D342B3429342B34293426342434D1
:100C40008134243426342B3429342834263428346F
:100C5000A93420346434693466344B34293428345C
:100C60002834283428342634283449342B346D343D
:100C70006434693466344B342934283428342834B5
:100C8000283426342834A9348034FF3FFF3FFF3F07
:100C9000FF3FFF3FFF3FFF3FFF3FFF3FFF3FFF3F64
:100CA000FF3FFF3FFF3FFF3FFF3FFF3FFF3FFF3F54
:100CB000FF3FFF3FFF3FFF3FFF3FFF3FFF3FFF3F44
:100CC000FF3FFF3FFF3FFF3FFF3FFF3FFF3FFF3F34
:02400E00753FFC
:08400000090012001300010089
:00000001FF
